:10000000B601092AB80071218413FA30A600A701AD
:10001000EE21A00AA50AA201A30100083805A60046
:10002000640000083805A7002606270538060319CE
:10003000A20A0319A30A2708A600A4030319A5030B
:100040000319A00B10282208042AB616B61EB612F1
:10005000B6192E28B6156920031855280830A300B4
:100060007E20A20DA30B3028B61E6020882084209D
:10007000B61A55205A2022080310042AB616B61EB6
:10008000B61236194828FE39B70036150310042A6F
:10009000361A5028A6003616692003185528260857
:1000A000712003185528B61E042A602088203611B6
:1000B0003612B6113A08840038088417800466287E
:1000C0003A08840038098005841780056728682865
:1000D000042A5A2088200822602084203708B61974
:1000E0000138A2000830A300A20D03185A20031CF7
:1000F000602088208420A30B74285A2088203A0886
:10010000840038080005FF3E3B0884003909632855
:100110003B08840039085D28A400B7172730A300E6
:1001200010309E200330A300E8309E20A3016430ED
:100130009E20A3010A309E202408A928A200250899
:10014000A1002408A000D2212008031DB713B71B6B
:100150000800303EA700071187108710831607118B
:1001600087108710F030860583122708B618D62826
:100170003A30A1009830AD213330A600EB20133087
:10018000A1008830AD21EB206430AC21EB2064303D
:10019000AC212230A600EB202830D5200C30D52011
:1001A0000630D520B6142708D6283614A600361CEB
:1001B000E4288710033C031CE928E9200730A1004C
:1001C000D030AD21031408003614FE3C0319042A74
:1001D0008714A60E361C36100715F0308605260843
:1001E0000F3986040711A60E3618EB283230AC21E1
:1001F00003140800B800841780048413A201201C93
:10020000A20008210319042A08210319042A082935
:100210003808A2060130A000A10100083805220616
:10022000031D0800A00A0319A10F0D290800A5014C
:10023000A400B7172730A30010302A210330A300F1
:10024000E8302A21A30164302A21A3010A302A219F
:1002500024083529A2002508A1002408A000D221E5
:100260002008031DB713B71B0800303EA6003A084C
:1002700084000930A70003104221A60CA70B3C29DB
:10028000031442298413B71D512900083804371D6F
:1002900038068000841700083804031C38068000E4
:1002A0005C2900083804031C38063719380680001A
:1002B0008417380980055C29370D0639A0006521AF
:1002C000A100A00A65210000AD2901308A002008A4
:1002D00082070134993403343934003460340C34E7
:1002E000FD3484178004042AA000A00DA00DA00DE9
:1002F0003830A005813020049F000030A10032304A
:10030000AD211F151F1982291E08A10083161E0882
:10031000042A03178D0083168C130C1483120C0807
:10032000042A03178C0083168C130C1555308D008E
:10033000AA308D008C148C189B290C11042AA3015F
:10034000A200FF30A207031CA307031C042A0330EA
:10035000A100E730AD21A129A101FC3EA000A10927
:10036000031CB829FF300000A0070318B329A00719
:100370006400A10FB2290800A2000130C229A20026
:100380000630C229A80023082102031DC92922081A
:100390002002043003180130031902302805031D20
:1003A000FF30042A1030A600A501A401210DA40DE0
:1003B000A50D2208A4022308031C230FA50203187D
:1003C000E8292208A40723080318230FA507031010
:1003D000A00DA10DA60BD6292008042A1030A800D4
:1003E000A101A001A70CA60C031CFC292208A00750
:1003F00023080318230FA107A10CA00CA50CA40C23
:10040000A80BF2292408042A83130313831264001F
:1004100008008316FF3085008E309F007030860004
:100420008113870183128601870107108316071045
:10043000643083129F218A112D2B86178316861311
:10044000FE308312AA200130AA202030AA202030BA
:10045000AA204830AA206530AA206C30AA206C302F
:10046000AA206F30AA202030AA202130AA200330F1
:10047000A300E830A021FE30AA200130AA20473096
:10048000AA203130AA204730AA203230AA20433097
:10049000AA203130AA205230AA205030AA20203081
:1004A000AA207630AA206530AA207230AA202E30E9
:1004B000AA203730AA202F30AA203230AA20363086
:1004C000AA200130A300F430A021FE30AA20C030C1
:1004D000AA20B130AA20B530AA202030AA206B3043
:1004E000AA206530AA207930AA202030AA207430B2
:1004F000AA206F30AA202030AA205330AA207430BE
:10050000AA206130AA207230AA207430AA20640088
:10051000061B872A08002C30A2000130A3000530FA
:10052000840020300220D4002308D50008000130C8
:10053000A000053084000230FA202008C6002108FF
:10054000C70008000130A000053084000430FA2004
:100550002008CA002108CB0008000130A0000530A7
:1005600084000830FA202008CE002108CF000800BF
:100570000130A000053084001030FA202008D2009D
:100580002108D300080000307421BC002108BD0000
:100590000A309F2108000730BA001030B800073039
:1005A000BB000830B900A03040203F0840203E0882
:1005B000402041084020400840203D0840203C08A1
:1005C0004020450840204408402049084020480871
:1005D00040204D0840204C08402051084020500841
:1005E0004020550840205408402041084020400841
:1005F0003E200A309F2108000730BA001030B800B2
:100600000730BB000830B900A03040203F08402030
:100610003E0840202720C1002720C0002720BD0021
:100620002720BC002720C5002720C4002720C900A0
:100630002720C8002720CD002720CC002720D1006C
:100640002720D0002720D5002720D4002720C10054
:100650002520C0000A309F210800861383168613C8
:1006600083121D22C8309F216400061F342BFE30E8
:10067000AA200130AA20B130AA20B530AA203A30F1
:10068000AA204C30AA206F30AA206730AA20203040
:10069000AA20B730AA202030AA203A30AA20503011
:1006A000AA206C30AA206130AA207930AA20FE301E
:1006B000AA20C030AA20B130AA20B630AA203A30F1
:1006C000AA204C30AA206F30AA206730AA20203000
:1006D000AA205330AA207430AA206F30AA2070308C
:1006E000AA20C8309F2164008A11061F8A2B8A1114
:1006F000861783168613323083129F2164008A1175
:10070000861E7A2C8A118613831686133230831242
:100710009F21732BD80164000A3058028A110318F4
:10072000A52B8A1186138316861383120130A3002A
:10073000F430A02186178316861383120130A3009C
:10074000F430A021D80A031D8B2BBE01BF013E0847
:10075000A0003F08A1000730A300CF30BC218A11C0
:10076000031D212C8A113E08A0003F08A100103073
:10077000A200A301D221B2002108B3000130320748
:10078000C00033080318013EC100C32297220310A2
:10079000460DC400470DC500A22203104A0DC80033
:1007A0004B0DC900AD2203104E0DCC004F0DCD00F6
:1007B000B8220310520DD000530DD1008B2203102C
:1007C000D40DD50DCB22FE30AA200130AA2041083D
:1007D000A50040088C203A30AA204508A50044080E
:1007E0008C203A30AA204908A50048088C203A30CD
:1007F000AA203D08A5003C088C20FE30AA20C0306D
:10080000AA204D08A5004C088C203A30AA20510897
:10081000A50050088C203A30AA205508A50054089D
:100820008C203030AA203030AA2064008A11061EA5
:10083000222C8A111030BE07031CA72BBF0A031DF0
:10084000A72B372B86138316861383120130A30040
:10085000F430A0213E08D7003E08A0003F08A100C8
:10086000A2010130A300D221D600031705308D006C
:10087000031357089121031706308D000313560800
:100880009121FE30AA200130AA205330AA207430D2
:10089000AA206F30AA207030AA204C30AA206F30D6
:1008A000AA206730AA206730AA206930AA206E30BB
:1008B000AA206730AA20FE30AA20C030AA204530E6
:1008C000AA204E30AA204430AA202030AA2054303A
:1008D000AA204930AA204D30AA204530AA203D3018
:1008E000AA204108A50040088C200B30A300B83096
:1008F000A021372B861783168613FE308312AA2079
:100900000130AA20B130AA20B530AA203A30AA205E
:100910005030AA206C30AA206130AA207930AA2059
:100920002030AA20B730AA202030AA203A30AA20AE
:100930005330AA207430AA206530AA207030AA2033
:10094000FE30AA20C030AA20B130AA20B630AA209A
:100950003A30AA204530AA204E30AA204430AA209E
:100960000330A300E830A02164008A11061FBF2CC9
:100970008A1164008A11861EB32D8A11B42C861345
:1009800083168613053083128921D700063089210A
:10099000D6005608A600A701A2010130A300EE214F
:1009A000B2002508B30057083207C2003308031805
:1009B000013EC300BE01BF013E08A0003F08A100E8
:1009C0000730A300CF30BC218A11031D6F2D8A117F
:1009D0003E08A0003F08A1001030A200A301D221D0
:1009E000B2002108B30001303207C00033080318F9
:1009F000013EC100FC220730BA004030B80002308E
:100A0000B7004108A500400818212C3036213D08C8
:100A1000A5003C0818213A3036214508A5004408B5
:100A200018212C3036214908A500480818212C30FF
:100A300036214D08A5004C0818212C3036215108CC
:100A4000A500500818212C3036215508A50054085F
:100A5000182130303621303036210D3036210A3021
:100A60003621FE30AA200130AA204108A500400806
:100A70008C203A30AA204508A50044088C203A3042
:100A8000AA204908A50048088C203A30AA203D0831
:100A9000A5003C088C20FE30AA20C030AA204D08BA
:100AA000A5004C088C203A30AA205108A500500817
:100AB0008C203A30AA205508A50054088C203030EC
:100AC000AA203030AA2064008A11061E742D8A11D3
:100AD0001030BE07031CDC2CBF0A031DDC2C0730C2
:100AE000A300D030A021372BFE30AA200130AA204D
:100AF0005330AA207430AA206F30AA207030AA2068
:100B00002030AA205030AA206C30AA206130AA20C0
:100B10007930AA206230AA206130AA206330AA204E
:100B20006B30AA20FE30AA20C030AA204530AA206F
:100B30004E30AA204430AA202030AA204430AA20D7
:100B40006130AA207430AA206130AA202330AA2064
:100B50003D30AA204108A50040088C200B30A3009E
:100B6000B830A021372B86138316861305308312E5
:100B70008921D70006308921D6005608A600A70192
:100B8000A2010130A300EE21B2002508B3005708EE
:100B90003207C20033080318013EC300BE01BF0183
:100BA0006400861ED02D3E08A0003F08A100430827
:100BB000A3004208BF218A11031DE12D8A11BE0145
:100BC000BF013E08A0003F08A1001030A200A30111
:100BD000D221B2002108B30001303207C00033082F
:100BE0000318013EC100FC220730BA004030B800B3
:100BF0000230B7004108A500400818212C303621EA
:100C00003D08A5003C0818213A3036214508A500CA
:100C1000440818212C3036214908A500480818211D
:100C20002C3036214D08A5004C0818212C303621D7
:100C30005108A500500818212C3036215508A50070
:100C40005408182130303621303036210D3036210D
:100C50000A303621FE30AA200130AA204108A50022
:100C600040088C203A30AA204508A50044088C2072
:100C70003A30AA204908A50048088C203A30AA201A
:100C80003D08A5003C088C20FE30AA20C030AA20D8
:100C90004D08A5004C088C203A30AA205108A50028
:100CA00050088C203A30AA205508A50054088C2002
:100CB0003030AA203030AA2064008A11861A6A2EA9
:100CC0008A111030BE020030031C013EBF02C83042
:100CD0009F21D32D64008A11061E7C2E8A11640088
:100CE0008A11061B7B2E8A111030BE070318BF0A1B
:100CF000C8309F21D32D5C2EFE30AA200130AA20BF
:100D00005330AA207430AA206F30AA207030AA2055
:100D10002030AA205030AA206C30AA206130AA20AE
:100D20007930AA206230AA206130AA206330AA203C
:100D30006B30AA200730A300D030A021372B6300EE
:020D40009F2EE4
:02400E00763DFD
:00000001FF
